:100000000EC015C014C013C012C011C010C00FC064
:100010000EC00DC00CC00BC00AC009C008C011241E
:100020001FBECFE5D1E0DEBFCDBF02D071C0E8CFAB
:10003000BC9AC49A80E197E228EC30E0F90131974C
:10004000F1F70197D9F7C49880ED97E028EC30E0FC
:10005000F9013197F1F70197D9F7C49A80E197E256
:1000600028EC30E0F9013197F1F70197D9F7C498FE
:1000700080ED97E028EC30E0F9013197F1F7019736
:10008000D9F7C49A80E197E228EC30E0F901319782
:10009000F1F70197D9F7C49880ED97E028EC30E0AC
:1000A000F9013197F1F70197D9F728EC30E0C49ABC
:1000B00080EA9FE0F9013197F1F70197D9F7C498E9
:1000C00080ED97E0F9013197F1F70197D9F7C49ADC
:1000D00080EA9FE0F9013197F1F70197D9F7C498C9
:1000E00080ED97E0F9013197F1F70197D9F7C49ABC
:1000F00080EA9FE0F9013197F1F70197D9F7C498A9
:1001000080ED97E0F9013197F1F70197D9F7CFCF5B
:04011000F894FFCF91
:00000001FF
